:100000000C9462000C94071A0C94341A0C948A0015
:100010000C948A000C948A000C948A000C948A0038
:100020000C948A000C948A000C948A000C948A0028
:100030000C948A000C94390B0C948A000C948A005E
:100040000C94611A0C948A000C94DD1D0C94201EF3
:100050000C948A000C948A000C948A000C948A00F8
:100060000C949A080C948A0000000007000201001A
:100070000003040600000000000000000102040864
:100080001020408001020408102001020408102002
:10009000040404040404040402020202020203032E
:1000A00003030303000000002300260029000000D2
:1000B0000000250028002B0000000000240027007D
:1000C0002A000E1F11241FBECFEFD8E0DEBFCDBF28
:1000D00012E0A0E0B1E0E0E9F0E402C005900D928A
:1000E000A03DB107D9F714E0A0EDB2E001C01D9228
:1000F000AA3BB107E1F710E0C4ECD0E004C02297BE
:10010000FE010E942320C23CD107C9F70E944A1F6A
:100110000C9446200C94000080910204813019F464
:1001200082E08093020480910204833019F484E019
:10013000809302040895A8950895CF93DF93FC015E
:10014000962F9270862F817060FF20C0992331F026
:1001500080914E0380831092D00216C0A091D002ED
:10016000C091E503C770D0E0C856DD4F8881A8175D
:1001700010F080E03CC081E08A0F8093D002B0E0B4
:10018000A250BD4F8C91808381E031C09923C1F092
:1001900090819093D1021092D002292F207E203698
:1001A00051F490914E03923020F390819F7190937F
:1001B000900393E01AC09E3F39F710924E0317C088
:1001C0009091D1029F3F01F79091D002993288F629
:1001D00021E0290F2093D0023081E92FF0E0E35491
:1001E000FC4F3083293281F691E090934E03DF91EA
:1001F000CF910895DC01ED91FC910190F081E02D0B
:1002000009950895DC01ED91FC910190F081E02DBC
:100210000995089560E08CE00E946F1B61E08BE01F
:100220000E946F1B61E08DE00E946F1B60E082E026
:100230000E946F1B61E084E00E946F1B089542E002
:1002400050E06CE870E080E00E94E7190895E3E078
:10025000F0E089E080935700E491E67081E0E630B9
:1002600009F080E00895CF93DF93C82F0E94270103
:10027000882381F0DFB781E080930104F8940E9425
:100280009B0088E180936000C0936000C1110E94D0
:100290009B00DFBFDF91CF9108952091BB03309188
:1002A000BC03382748E0C901880F991F37FF06C0F3
:1002B0009C0151E2252750E1352701C09C014150A6
:1002C00091F73093BC032093BB030895D82FC0E06F
:1002D000CD1780F45E9A64E670E080E090E00E94C2
:1002E000DA1A5E9864E670E080E090E00E94DA1A24
:1002F000CF5FEECF6CE271E080E090E00E94DA1A0E
:10030000E6CF0F931F93CF93DF93EC01062F15E0F9
:10031000115051F0CE010E943020081741F0602F9B
:10032000CE010E943820F4CF82E00E946601DF9166
:10033000CF911F910F910895A0E0B0E0E2EAF1E0C3
:100340000C94EC1F482E562EC0E0D0E0612C712C8E
:10035000E12CF12C00E010E0442079F081E0481617
:10036000A1F092E0491219C078E4672E712CE0E206
:10037000EE2EF12C01E513E010C0612C712CBBE1D5
:10038000EB2EF12C06EE13E008C0FDE16F2E712C70
:10039000A9E2EA2EF12C0DEB13E043018C0E9D1E19
:1003A0001092BC031092BB033401A62CA818B12CE8
:1003B000C30101966C01AE14BF04A8F4A00EB11ED7
:1003C000511006C0C3010E943020F501808305C092
:1003D000F5016081C3010E948101F50180810E94C5
:1003E0004D013601E2CFC301511018C0C3010E9474
:1003F0003020B82EC6010E9430202B2D30E0322F45
:100400002227282B8091BB039091BC03821793076E
:1004100079F4C0E0D0E0552453949ECF360160912A
:10042000BC030E9481016091BB03C6010E9481014F
:10043000D395C13093E0D90708F48ECF852DCDB781
:10044000DEB7E0E10C94082060E081E00E949C01AE
:10045000882331F081E09091BD03973309F080E06B
:10046000089561E081E00E949C0108958436910521
:1004700020F4BC0180E090E017C09C018E3B910508
:1004800028F42A553109AAE0B0E00CC0823D91055C
:1004900028F4245B3109A4E6B0E004C02D5C3109E6
:1004A000A8E5B2E00E94571FA4E6B0E09B01AC01B2
:1004B0000E94661F089590E08C599F4F0E9436025B
:1004C000089561E082E00E949C01089560E082E06E
:1004D0000E949C01811106C08FEF9FEF9093520301
:1004E00080935103089595E09093E60390E29093F2
:1004F000E70392E29093E80391E29093E90393E299
:100500009093EA039BE29093EC0394E29093ED03C3
:1005100095E29093EE0392E09093F4039FEF909313
:10052000F5039AE09093FE031092FF0310920004EB
:100530001092F6031092F7031092F8031092F90349
:100540002EE12093FA039093FB0328EB3BE03093DA
:10055000FD032093FC03882361F061E080E00E94AA
:100560009C018FEF9FEF90935203809351030E9461
:100570006102089560E080E00E949C01811103C047
:1005800081E00E9473020895FC0140A5842F8770CA
:1005900090E0959587950196242F217030E0820F89
:1005A000931F880F880F08958F929F92AF92BF92EA
:1005B000CF92DF92EF92FF92CF93FC01C0A5EC2F78
:1005C000E770F0E0E856FD4FA081B0E0C7FF03C040
:1005D00024E130E002C02FE030E0FC0197A183E18C
:1005E000989FF0011124E25CFE4F80809180A280F0
:1005F000B380A20FB31F20E43FE14DE750E00E941B
:10060000711FA50194010E94A91F8C2F887149F4C4
:1006100069017A01E0EDCE0EE7E0DE1EE11CF11C7F
:100620001BC0C7FF05C060E47AE88CE29EE004C00E
:1006300060E07EEE8AEB9BE069017A01F8EBCF0E79
:10064000FBE0DF1EE11CF11CA50194010E94A91F23
:10065000C20ED31EE41EF51EC701B60169517C4FC0
:100660008F4F9F4F28EE33E040E050E00E94A91FDB
:10067000A8EEB3E00E94661FCF91FF90EF90DF904D
:10068000CF90BF90AF909F908F900895DB01FA01BB
:10069000582F569590E02481237030E0322F222786
:1006A0004081240F311D11963C932E9344814C7050
:1006B000218130E060E4469F200D311D1124139606
:1006C0003C932E93129744814073228130E060E185
:1006D000469F200D311D112415963C932E9314979F
:1006E0004481407C238130E064E0469F200D311D31
:1006F000112417963C932E931697359618969F5F64
:10070000591748F680FF47C0408142954695469567
:1007100043702DE431E0429FC001439F900D1124AE
:100720000C9611969C938E93808190E044E0969570
:1007300087954A95E1F783709927829FA001839F4F
:10074000500D929F500D1124445F5F4F13965C93A0
:100750004E931297808190E0969587959695879510
:1007600083709927829FA001839F500D929F500D07
:100770001124445F5F4F15965C934E93149740810C
:100780004370429FC001439F900D11240C96179611
:100790009C938E9316970895803223E0920708F178
:1007A000883E23E0920740F48F519340E4E0969511
:1007B0008795EA95E1F70895803D27E0920718F4C0
:1007C0008C5D93400895883928E0920768F4885C2E
:1007D000974074E0969587957A95E1F78D509C4FF8
:1007E000089580E090E008958FEF93E008958C30B5
:1007F000910540F4A4E0880F991FAA95E1F7885D60
:100800009C4F0895843F23E0920718F484529C4F34
:100810000895811524E0920740F48657934FF4E041
:10082000880F991FFA95E1F7089580E998E00895F7
:100830009C013695279525753575821B930B9C0178
:1008400023733373969587959695879583739373E2
:10085000820F931F9C0154E0369527955A95E1F736
:10086000280F391F2F703F7041E051E0249FC001D5
:10087000259F900D349F900D1124892F08952D9858
:10088000882319F000002B9A02C000002B9800006A
:100890002D9A000008952D9A000083B12D98000034
:1008A000829581700895CF93DF93D82F5C9A2D980D
:1008B0005C98C8E08D2F80780E943F04DD0FC15006
:1008C000C9F72D98DF91CF9108958F770E94530437
:1008D0000895CF93DF93D82FC8E08D2F80780E94A2
:1008E0003F04DD0FC150C9F72D98DF91CF910895D6
:1008F000CF93DF932D98C8E080E0D82FDD0F0E94C2
:100900004B048D0FC150C9F7DF91CF9108950E941C
:1009100065040E9478045C9A0895A1E0B0E0E3E9E0
:10092000F4E00C94FA1F806869830E945304698183
:10093000862F0E9469045C9A2196E2E00C941620AE
:10094000CF93C091C603C827E82FF0E0E354FC4FD3
:10095000678589E70E948D046C2F8DE30E948D04CA
:100960006C2F82E40E948D04CF91089586E20E944C
:1009700087040895CF938BE20E948704C82F8CE2EE
:100980000E948704282F30E066E0369527956A9507
:10099000E1F744E0C49FC0011124822B932BCF9137
:1009A0000895CF93DF93EC016C818CE10E948D045C
:1009B0006D818DE10E948D046E818EE10E948D0417
:1009C0006F8180E20E948D04688581E20E948D041F
:1009D000698582E20E948D046A8583E20E948D040B
:1009E0006B8584E20E948D046C8585E20E948D04F3
:1009F0006D858AE20E948D046E858EE60E948D04CC
:100A00006F858FE60E948D04688980E70E948D04BF
:100A1000698981E70E948D046A8982E70E948D04BA
:100A2000DF91CF910895CF92DF92EF92FF92CF9313
:100A3000DF936B017C01C11488E3D8068CE9E806DA
:100A40008CE1F80628F5C701B60120E836E948E947
:100A500050E00E94A91FE901689760E879E687E6FF
:100A60009FEF0E94791F6C0D7D1D8E1D9F1DF2E072
:100A7000660F771F881F991FFA95D1F721E732E09B
:100A800040E050E00E94A91FF22EE32E80E421C036
:100A9000C701B60120E03DE241E351E00E94A91FF9
:100AA000E901689760E073ED8EEC9EEF0E94791F7C
:100AB0006C0D7D1D8E1D9F1D660F771F881F991F52
:100AC00021E732E040E050E00E94A91FF22EE32E21
:100AD00080E66C2F6F71680F85E70E948D046E2D84
:100AE00086E70E948D046F2D87E70E948D04DF91B9
:100AF000CF91FF90EF90DF90CF9008958F929F92CB
:100B0000AF92BF92CF92DF92EF92FF92CF93DF939B
:100B1000D82F83E00E9487048093BA0384E00E9468
:100B200087048093B90360E086E00E948D0461E051
:100B300087E00E948D046FE789E00E948D0465E0E4
:100B40008AE00E948D0462E18BE00E948D0465E1E1
:100B50008CE00E948D046DEF8DE00E948D0460E0BA
:100B60008EE00E948D04DD2319F08BE291E008C035
:100B70002091E40333E1239FC0011124825C9E4F46
:100B80000E94D1046CE880E30E948D046FE082E350
:100B90000E948D0462E483E30E948D048091E5034A
:100BA00087FF02C064E101C06AE084E30E948D0413
:100BB0006AE285E30E948D046DE286E30E948D0463
:100BC00064ED87E30E948D0460E088E30E948D0459
:100BD00060E089E30E948D04D11109C0C090C60372
:100BE000D090C703E090C803F090C90307C0C5E8E0
:100BF000CC2EC1ECDC2EED2CCEEDFC2ECAE38F2CDE
:100C00009924AA24BB24682D8C2F0E948D04682D62
:100C100085E08C0F0E948D04FE2CED2CDC2CCC2466
:100C2000CF5FCE3361F76FEF83E40E948D046FEFE7
:100C300084E40E948D046FEF85E40E948D046FEFC1
:100C400086E40E948D04DD2311F066E002C060910D
:100C5000CA038DE60E948D0460E089E70E948D043E
:100C60006091CB038AE70E948D0460E083E70E94D5
:100C70008D0460E084E70E948D04D11109C0609169
:100C8000C2037091C3038091C4039091C50304C053
:100C900060E071EA8CEB93E30E941305DF91CF9142
:100CA000FF90EF90DF90CF90BF90AF909F908F908C
:100CB000089561E087E00E948D0464E28EE70E945F
:100CC0008D0463E088E00E948D0460E088E00E946B
:100CD0008D0465E087E00E948D0462E085E00E945B
:100CE0008D0483E00E9487048093BA0384E00E940D
:100CF00087048093B903089583E00E94870480935A
:100D0000BA0384E00E9487048093B90361E087E01E
:100D10000E948D046AE070E080E090E00E94DA1AA0
:100D20000E94590600000895CF92DF92FF920F9320
:100D30001F93CF93DF931F92CDB7DEB7082F162FE7
:100D40008EE399830E948D04F02EC02E9981D92EB6
:100D50008C2D8F19811738F4F60161916F018FE79F
:100D60000E948D04F5CF64E085E00E948D0483E04D
:100D70000E9487048093BA0384E00E9487048093D2
:100D8000B9030E94B71A6093B5037093B6038093BA
:100D9000B7039093B80369E087E00E948D0481E077
:100DA000809302040F90DF91CF911F910F91FF90DC
:100DB000DF90CF9008950F931F930E949406809127
:100DC0000204813099F40E94B71A0091B503109182
:100DD000B6032091B7033091B803601B710B820BEF
:100DE000930B603A76488140910548F38091020464
:100DF000813031F46CEB71E080E194E00E94791C69
:100E00001F910F9108950F931F93809102048230D8
:100E100021F41092020481E020C08091020481300C
:100E2000D9F40E94B71A0091B5031091B60320912E
:100E3000B7033091B803601B710B820B930B613ABF
:100E400076488140910540F061E087E00E948D0482
:100E50001092020482E001C080E01F910F9108957A
:100E6000EF92FF920F931F93CF93DF938B019C011F
:100E7000442737FD4095542F60E271EA87E090E007
:100E80000E94CB1FE9011C161D0614F0C1E0D0E042
:100E9000D80120E231EA47E050E00E94711F9E0134
:100EA000442737FD4095542F0E94CB1F790100E065
:100EB00010E00E151F055CF42B9ACE010E94001B5A
:100EC0002B98CE010E94001B0F5F1F4FF2CFCDB7B2
:100ED000DEB7E6E00C941220CF93C82F5D9A83E032
:100EE0000E9487048093BA0384E00E948704809361
:100EF000B90360E086E00E948D0461E087E00E9413
:100F00008D046FE789E00E948D0465E08AE00E940D
:100F10008D0462E18BE00E948D0465E18CE00E940B
:100F20008D046DEF8DE00E948D0460E08EE00E94E4
:100F30008D046CE280E70E948D0460E080E30E94F3
:100F40008D0460E089E70E948D0465E08AE70E94D5
:100F50008D0462E181E70E948D0462E082E70E94D5
:100F60008D0460E083E70E948D0460E084E70E94C6
:100F70008D046091F6037091F7038091F8039091CE
:100F8000F9030E94130567E08DE60E948D046AE074
:100F900070E080E090E00E94DA1A69E087E00E9449
:100FA0008D046AE070E080E090E00E94DA1ACC23C1
:100FB00069F0C5E1C15009F459C061E070E088EB07
:100FC00091E00E9430070E949B00F4CF61E070E046
:100FD00088E891E00E9430070E949B0065E08DE662
:100FE0000E948D046AE070E080E090E00E94DA1ACE
:100FF00061E070E088EB91E00E9430070E949B0066
:1010000064E08DE60E948D046AE070E080E090E08C
:101010000E94DA1A61E070E08DE591E00E943007ED
:101020000E949B0062E08DE60E948D046AE070E001
:1010300080E090E00E94DA1A61E070E08FEA90E0D0
:101040000E9430070E949B0060E08DE60E948D04A4
:101050006AE070E080E090E00E94DA1A62E070E0FE
:1010600085E091E00E9430070E949B0061E087E0EC
:101070000E948D045D98CF910895CF93DF93EC018A
:101080004AE050E06D2F70E080E194E00E943E1D48
:101090006EE280E194E00E945D1CBE0184E07695E2
:1010A00067958A95E1F76F7077274AE050E080E115
:1010B00094E00E943E1D6EE280E194E00E945D1C7F
:1010C000BE016F7077274AE050E080E194E00E9413
:1010D0003E1DDF91CF910895CF93C1E0811101C0F2
:1010E000C0E06C2F82E10E94A81B6C2F83E10E945C
:1010F000A81B1092AF031092AE038091B9008C6FC1
:101100008093B90080E28093B80085E48093BC00AE
:10111000CF91089585ED8093BC008091BC0084FD43
:10112000FCCF0895ECEBF0E0108285E48083109210
:10113000AE0308951F920F920FB60F9211242F93B2
:101140003F934F935F936F937F938F939F93AF934F
:10115000BF93EF93FF93CF93DF931F92CDB7DEB78B
:101160008091B900887F803609F4C7C0A8F588321D
:1011700009F464C098F4803109F45DC038F4882320
:1011800009F4F3C0883009F456C0F1C0883109F47D
:1011900055C0803209F0EBC082E0A7C0803409F46A
:1011A00077C078F4803309F45FC0883309F0DFC07A
:1011B00084E08093AD038091AE038B7F8093AE0378
:1011C000D0C0803509F452C0883509F467C088342E
:1011D00009F0CDC085E089C0883909F4C0C0A8F401
:1011E000883709F48AC038F4883609F486C0803715
:1011F00009F483C0BCC0883809F4B1C0803909F44F
:101200007FC0803809F0B3C07BC0803B09F493C035
:1012100038F4803A09F48CC0883A09F48CC0A7C02D
:10122000803C09F49EC0883C09F49BC0883B09F0CF
:101230009EC080E081C08091B20313C08091AF0353
:101240009FEF980F9093AF038823D1F1E091B00303
:10125000F091B103CF0101969093B1038093B00355
:1012600080818093BB007DC083E03FC0E091B003EC
:10127000F091B103CF0101969093B1038093B00335
:101280008091BB0080838091AF0381508093AF0336
:101290008091AF03823008F064C061C0E091B00378
:1012A000F091B103CF0101969093B1038093B00305
:1012B0008091BB0080838091AF0381508093AF0306
:1012C0008091AE038B7F8093AE038091AE0380FF4D
:1012D0004CC08091AE038E7F8093AE038091AE03AD
:1012E00082608093AE0384EA3DC08093AD03809119
:1012F000AE038B7F8093AE0338C01092AF0331C032
:10130000E091B303F091B403309749F18091BB00B1
:1013100089838091AF0391E0980F9093AF0381117F
:1013200002C062E001C060E0CE010196099515C0DF
:101330000E948A0816C081E0E091B303F091B403E3
:10134000309769F0882311F063E001C061E0CE01BD
:101350000196099599819093BB00811102C085E89F
:1013600001C085EC8093BC0002C00E948A080F90E7
:10137000DF91CF91FF91EF91BF91AF919F918F91AD
:101380007F916F915F914F913F912F910F900FBE81
:101390000F901F9018958F929F92AF92BF92CF920D
:1013A000DF92EF92FF92CF93DF93EC010E94B71A86
:1013B0006B017C014E01A12CB12C8091AE0382FF08
:1013C00011C02097D1F30E94B71A6C197D098E09BC
:1013D0009F0986169706A806B90678F70E94920814
:1013E00081E004C08091AD031092AD03DF91CF91F5
:1013F000FF90EF90DF90CF90BF90AF909F908F9035
:101400000895A2E0B0E0E7E0FAE00C94F61F182F90
:101410007B01022F047022FD05C08091090190918B
:101420000A0102C080E090E02A8349830E94CB0930
:101430002A814981811136C01092AD034093AF03D8
:10144000F092B103E092B003110F1093B2039091A8
:10145000AE0321FF02C085E001C084E0892B8093A8
:10146000AE038091AE0381FF0BC08091AE038D7FF0
:101470008093AE038091B2038093BB0085EC01C0E2
:1014800085EE8093BC00822F817020FF0BC001117C
:1014900005C08091090190910A0102C080E090E0AE
:1014A0000E94CB092296E6E00C941220A2E0B0E064
:1014B000ECE5FAE00C94F61F182F7B01022F047064
:1014C00022FD05C08091090190910A0102C080E0CF
:1014D00090E02A8349830E94CB092A8149818111A6
:1014E00038C01092AD034093AF03F092B103E09285
:1014F000B003812F880F81608093B2039091AE0377
:1015000021FF02C085E001C084E0892B8093AE03F7
:101510008091AE0381FF0BC08091AE038D7F8093DD
:10152000AE038091B2038093BB0085EC01C085EED1
:101530008093BC00822F817020FF0BC0011105C079
:101540008091090190910A0102C080E090E00E9420
:10155000CB092296E6E00C941220A0E0B0E0E3EB89
:10156000FAE00C94F41F0E94B71A0091A90310919D
:10157000AA032091AB033091AC036B017C01C01A2C
:10158000D10AE20AF30A9701860141E1C41647E253
:10159000D406E104F10408F442C02091A80331E02C
:1015A000320F3093A80320FF02C017E001C010E003
:1015B0006093A9037093AA038093AB039093AC0349
:1015C00063E070E080E194E00E94020161E070E07D
:1015D00080E194E00E94020107E0010F812F90E07A
:1015E000EC01CC0FDD1FC55FDE4F68817981672F6D
:1015F000772763707727880F991F880F991F682BAB
:10160000792B80E194E00E94FA0068817981772744
:1016100080E194E00E94FA001F5F1013DFCFCDB786
:10162000DEB7E8E00C94102025B190E0FC01EE0F4D
:10163000FF1FE80FF91FE85EFC4F8081282B25B9BA
:1016400088B19181892B88B98BB19281892B8BB913
:10165000089585B190911503892385B988B190913A
:101660001603892388B98BB19091170389238BB90D
:1016700008951F920F920FB60F9211242F933F934C
:101680004F935F936F937F938F939F93AF93BF938A
:10169000CF93EF93FF93C091740380910601C81715
:1016A00008F03EC08091130390911403909387003B
:1016B00080938600EC2FF0E0EE0FFF1FE55FFE4FFA
:1016C000808191810E94F703880F991F90931403E2
:1016D00080931303809113039091140320910701C9
:1016E00030910801281B390B309308012093070122
:1016F0008091FC039091FD03880F991F28173907EB
:1017000020F4909308018093070180917203811166
:1017100042C08091F40380FF41C0C830E0F53EC074
:101720008091130390911403909387008093860017
:101730008091070190910801909314038093130303
:1017400080917203882319F08FEF9FEF06C080917C
:1017500013039091140388559240909389008093CD
:10176000880080E49CE990930801809307018091B0
:101770008400909185008097D0F30E94290B80917E
:101780007303811105C08091060181500E94140BE2
:101790001092740327C08FEF9FEF06C08091130350
:1017A000909114038855924090938900809388000B
:1017B00080918400909185008097D0F30E94290B3E
:1017C00080917303811104C080917403811106C05C
:1017D000809174038F5F8093740304C081500E94D2
:1017E000140BF6CFFF91EF91CF91BF91AF919F91E5
:1017F0008F917F916F915F914F913F912F910F90BA
:101800000FBE0F901F90189524E0829FC0011124F5
:101810008C30910538F0853F23E0920728F084EF63
:1018200093E008958CE090E00895CF93DF93C0910A
:10183000F503C03390F48C2F807339F0803141F47C
:10184000809175038295807F05C080917A0302C0E4
:1018500080917B03CF70D0E015C0CF33E0F4CF7020
:10186000D0E0809175038295807F0E94040CDE0198
:10187000AA0FBB1FA55FBE4F11969C938E93219616
:1018800080917B030E94040CFE01EE0FFF1FE55FB9
:10189000FE4F91838083DF91CF91089580917603ED
:1018A000909177039F770E941804809375038F307F
:1018B00029F480917B038695805804C099E0899F24
:1018C000802D112480937A03F8940E94150C78944B
:1018D0008091E9038132E1F480917A039FEF980FC0
:1018E0009E3F78F08091B0008F7D8093B00061E0E2
:1018F00080917A03811101C060E083E00E94A81BFF
:1019000008958093B4008091B00080628093B0000D
:101910000895FF920F931F93CF93DF9307EE13E089
:10192000C0E0D0E0B3E0FB2E8C2FD801ED918D010B
:101930009E2F907F9031F1F4EF70F0E0EE0FFF1FDB
:10194000E55FFE4F208131816F2D0E94891FE92FB5
:10195000F0E0EE0FFF1FEE56FD4F61E080819181B8
:101960008217930708F060E0FE01E056FD4F80818A
:101970000E94A81B2196C830D105B1F6CDB7DEB7BD
:10198000E5E00C941320809151039091520301964D
:1019900031F1E1E5F3E080E090E04091F503242FA0
:1019A0002F7030E08217930799F02F5F3F4F821717
:1019B000930711F4403360F4F89420813181DC0105
:1019C000AA0FBB1FA55FBE4F11963C932E93789430
:1019D000019632968031910501F70E94890C089595
:1019E000FF920F931F93CF93DF938DEB93E00E94B1
:1019F000C402809306019091F503292F2F702813BC
:101A000004C081E0820F8093060190539F3060F400
:101A10004091060130E0842F90E0019728173907A4
:101A200019F44F5F4093060180910601813118F04F
:101A300080E180930601EAE1F3E0DF0112971C9256
:101A4000DF0111971C921082339623E0E233F207F4
:101A5000A1F74FEF3FEFAAEAB2E007EE13E02FEF56
:101A6000E80189918E018031F8F490E0FD01329710
:101A70006081FC01EE0FFF1FE80FF91FE85EFC4FCD
:101A80008081862B8083CD010197EC015881818173
:101A9000852B81839C918281892B828360955095CF
:101AA00090952923352346231396D3E00F3E1D0737
:101AB000B9F6409315033093160320931703C0EA39
:101AC000D2E007EE13E0F12CF80181918F01823210
:101AD00030F08632B8F0863211F460E010C0F6E0E3
:101AE000FF1204C08091C1008F7E06C027E0F21271
:101AF00005C08091C100877F8093C10061E088812B
:101B00000E946F1BF394219688E0F812DDCF80913C
:101B1000E703803231F461E089E00E94A81B82E88B
:101B200001C082E08093800081E080937303809302
:101B300072038091E903813211F08732D9F461E0B8
:101B400083E00E946F1B60E083E00E94A81B8091ED
:101B5000E903813231F481E08093B0008093B100D9
:101B600009C082E08093B00085E08093B1008EE3ED
:101B70008093B3008AE1809381008FEF9FEF909371
:101B800089008093880080ED97E090938700809390
:101B9000860080E49CE9909308018093070190936C
:101BA0001403809313031092740380916F0081607B
:101BB00080936F008091F40383FF0CC080915103E8
:101BC00090915203019631F00E94C30C109272035F
:101BD00010927303CDB7DEB7E5E00C941320CF93DA
:101BE000C82F8091EC038B3221F46C2F8FE00E9480
:101BF000A81B8091E903873249F48091B000CC237F
:101C000011F0806101C08F7E8093B000CF91089564
:101C1000A5E2B0E0EEE0FEE00C94EA1F6B017C016F
:101C20000E94AB1A4B015C0181E00E947E0583E0BB
:101C3000809302040E947C0668EC71E080E194E0ED
:101C40000E94791C44244A94542CF6E42F2EA5E5D6
:101C50003A2EC114D104E104F10469F00E94AB1AD8
:101C6000681979098A099B096C157D058E059F0500
:101C700010F080E0E5C080910204843051F766EDF9
:101C800071E080E194E00E94791C8FE70E94650476
:101C90000E9478048CA3823601F50DEB13E00E94BC
:101CA0007804F80181938F01F3E0063E1F07B9F72E
:101CB0008091BD03873309F0BDC06FED71E080E115
:101CC00094E00E94791C82E48CA361E0CE018496AA
:101CD0000E94DB065D9A81E0B3C0803741F089360F
:101CE00019F581E00E94730289E4898305C020E52B
:101CF0002983C12CD12C7601909101048091F403A9
:101D0000992311F0806801C08F778093F403E6EE89
:101D1000F3E0DE0112968BE101900D928A95E1F7D6
:101D20006CE1CE01019684C08437D9F494E599839F
:101D300093E09A838B8388E08C838FE08D838EE1A0
:101D4000EDE9F1E0DE01169601900D928A95E1F73A
:101D500063E2CE0101960E94DB06C12CD12C7601F4
:101D600069C0853789F406EE13E00E947804F80113
:101D700081938F01F4E001301F07B9F761E080E043
:101D80000E949C013CA251C0863629F52091510346
:101D9000309152032F3F3F4FD9F0298271E5672ED2
:101DA00073E0772E8E010D5F1F4FF30181919191AA
:101DB0003F010E94F703F80131979083F801808377
:101DC0000E5F1F4FF1E76F16F3E07F0671F701C05A
:101DD000898361E2A6CF8736E9F401E513E00E942A
:101DE0007804682E712C762C66240E947804930166
:101DF000280F311DC9010E94CC03F80181939193F2
:101E00008F01F3E001371F0751F727E42CA30E944D
:101E100061020BC0873471F4509252034092510317
:101E20008DA30E9461028DA18CA361E0CE018496F6
:101E30000E94DB0683E0809302040E94590609CFCA
:101E4000A596E2E10C9406201F93CF93DF93C82F51
:101E5000D62F61E00E946F1B61E08C2F0E94A81BAF
:101E600061E08D2F0E94A81B8AE090E00E94001B79
:101E70008D2F0E94DB1B892B71F060E08C2F0E945C
:101E8000A81B8AE090E00E94001B8D2F0E94DB1BA4
:101E900011E0892B09F010E060E08C2F0E946F1B8D
:101EA00060E08C2F0E94A81B60E08D2F0E94A81B71
:101EB000812FDF91CF911F91089580E48093BA0024
:101EC0001092BD008DE990E09093B4038093B3032A
:101ED00010924E0315E004E0B2E0FB2E80914E0319
:101EE000813039F480E00E947E05F0924E035E98C6
:101EF000F5CFC0914E03C33061F45D98809190039B
:101F00000E94A004C09302040E94590600934E034D
:101F1000E5CF80914E03843009F78091020484302C
:101F2000E9F68FE70E946504CEEFD2E0E091E50389
:101F3000E770F0E0E856FD4F808190E09E012E5F53
:101F400032402817390724F40E9478048993EECF91
:101F500010934E035D9AC2CFAAE2B0E0E2EBFFE03D
:101F60000C94F91F1FEF198389E2EDEBF3E0DE011A
:101F7000129601900D928A95E1F721E04AE2BE01A6
:101F80006F5F7F4F80E20E94010A81110EC021E045
:101F900041E0BE016F5F7F4F80E20E94560A8111CF
:101FA00004C082E080934E0302C010934E038091E0
:101FB0004E03823051F00E94AB1A60934A03709333
:101FC0004B0380934C0390934D03AA96E3E00C944B
:101FD0001520A1E0B0E0EFEEFFE00C94FA1F809135
:101FE0004E038230D9F480919003805A898321E096
:101FF00041E0BE016F5F7F4F80E20E94010A8823AB
:1020000069F08FEF80934E030E94AB1A60934A03EE
:1020100070934B0380934C0390934D032196E2E021
:102020000C941620A1E0B0E0E8E1F0E10C94FA1F76
:1020300080914E038230D1F421E041E0BE016F5F18
:102040007F4F80E20E94560A882371F08FEF8093C1
:102050004E030E94AB1A60934A0370934B03809324
:102060004C0390934D0302C0898101C08FEF2196EC
:10207000E2E00C941620A2E2B0E0E1E4F0E10C947E
:10208000EA1F9E012F5F3F4F80E1D9011D928A9583
:10209000E9F76AEE71E080E194E029A33AA30E9497
:1020A000791C0E947C061D8A1E8A1F8A188E312C7C
:1020B000212C00E0812C912C5401412C84E7582ED6
:1020C0008BE8682E82E3782E90E5C92E93ECD92E0A
:1020D000E12CF12C84EF91E0A0E0B0E08D8F9E8F99
:1020E000AF8FB8A380E09EECADEEB4E3898F9A8FFA
:1020F000AB8FBC8F80E094E7ABE8B2E3898B9A8B1F
:10210000AB8BBC8B80E194E00E94451D892B09F4C8
:10211000E1C080E194E00E94721D9C0133272C32C3
:10212000310509F442C0ACF42332310509F0ABC0EB
:1021300019821A821B821C821D821E821F821886AF
:1021400019861A861B861C861D861E861F86188A7F
:1021500060C02434310529F02335310509F4B2C0BB
:1021600092C064E480E194E00E945D1C2AE030E0CB
:1021700040E054E76BE872E380E194E00E94D91CF0
:102180006CE280E194E00E945D1C2AE030E040E0D7
:102190005EEC6DEE74E380E194E00E94D91C6CE289
:1021A00080E194E00E948B1CADCF0F5F043009F0FA
:1021B000A9CF29813A814B815C81A8EEB3E00E94CE
:1021C000661F698B7A8B8B8B9C8B2D813E814F8117
:1021D00058850E94661F698F7A8F8B8F9C8F298507
:1021E0003A854B855C852D8F3E8F4F8F58A32D856B
:1021F0003E854F8558890E94661F6B017C016032C5
:102200003EE473078105910530F462E38CE10E949E
:102210008D0400E077CF603345E7740781059105B1
:1022200010F462E2F3CF60345CE975078105910533
:1022300010F466E2EBCF80E5C81683ECD806E10423
:10224000F10410F462E1E2CF90E6C9169AEED906E5
:10225000E104F10410F465E1D9CFA0E7CA16A1E1C9
:10226000DA06A1E0EA06F10410F461E0CFCFB0EAAB
:10227000CB16B6E8DB06B1E0EB06F10410F463E040
:10228000C5CF65E0C3CF10ED180F1A3008F03ACF74
:10229000E1E0F0E0EC0FFD1F24E0029FE00DF11DF6
:1022A00011242081318142815381AAE0B0E00E9453
:1022B000661F610F711D811D911D60837183828373
:1022C000938320CF49885A886B887C88812C912CF5
:1022D000540118CF81149104A104B10489F4C301FD
:1022E000B2010E94130561E070E080E090E00E947E
:1022F000DA1A1D8A1E8A1F8A188E312C22242A94EB
:102300008D8D9E8DAF8DB8A188169906AA06BB0645
:10231000D0F40E94B6042D893E894F89588D280F2C
:10232000311D411D511D2D8B3E8B4F8B588F381603
:1023300008F4382E821508F4282E3FEF831A930AEA
:10234000A30AB30A56C0C301B20128EE33E040E04D
:1023500050E00E94A91FBA01A9012AE030E080E103
:1023600094E00E94271D6CE280E194E00E945D1CD5
:102370004AE050E0632D80E194E00E94361D6CE25B
:1023800080E194E00E945D1C6D897E898F89988D23
:10239000A50194010E94A91FBA01A9012AE030E019
:1023A00080E194E00E94271D6CE280E194E00E94AD
:1023B0005D1C4AE050E0622D80E194E00E94361DF1
:1023C0006CE280E194E00E948B1C4C0C5D1C6E1C46
:1023D0007F1C898D9A8DAB8DBC8D84159505A605C6
:1023E000B70520F449885A886B887C88812C912C09
:1023F000540129893A894B895C89283E334041053B
:10240000510509F07FCEA296E2E10C940620A1E0EE
:10241000B0E0EDE0F2E10C94FA1F80E00E9433019D
:1024200061E085E00E946F1B61E086E00E946F1B07
:102430000E940A0160E080E00E946F1B61E081E081
:102440000E946F1B40E052EC61E070E080E194E09C
:102450000E948D1E0E94BA020E94660267EF71E020
:1024600080E194E00E945A1C84E793E00E943D08BA
:102470006EE072E080E194E00E945A1C4AE050E075
:1024800067E070E080E194E00E940F1D0E941F0150
:1024900078945E9A63E183E00E94240F882329F0F8
:1024A0005E985D980E943B10FBCF62E189E00E943C
:1024B000240F811104C00E942402811119C061E51A
:1024C00072E080E194E00E945A1C60E070E0CB0171
:1024D0000E94080E882349F00E94310266E172E0F2
:1024E00080E194E00E94791C5D9A0E94F00C10C07B
:1024F0000E94F00C8091E803823209F0CAC08091FA
:10250000EA03833209F0C5C08091F40381FDC7C09E
:102510008091E803823231F58091EA03833211F52C
:1025200081E00E946C088091F40382FF08C061E39F
:1025300072E080E194E00E94791C0E945D0F64E1EA
:1025400070E080E090E00E94DA1A21E041E0BE01F4
:102550006F5F7F4F80E20E94560A811103C081E0C5
:1025600080934E036CE372E080E194E00E945A1C79
:102570008FE00E94330180E00E947E05109290035C
:1025800080E00E94A00480E0883170F08093D20245
:1025900083E0809302040E947C0680914E0388238E
:1025A00071F00E94AC0F0BC021E0280FE82FF0E083
:1025B000E354FC4F9785992349F3822FE5CF80910F
:1025C000EE03982F9D7F983229F440E052EC61E0B1
:1025D00070E027C0893271F440EA56E861E070E0AB
:1025E00080E194E00E948D1E8091C2008062809301
:1025F000C2001BC08091E5038871803129F440E856
:1026000055E260E070E00DC04091BE035091BF0301
:102610006091C0037091C1034A3051056105710595
:1026200070F380E194E00E948D1E80E194E00E94AE
:10263000451D892B29F080E194E00E94721DF5CFA1
:102640008091ED03843229F08091C1008F7E8093C8
:10265000C1008091EE03853241F08852833028F02A
:102660008091C100877F8093C1001092D4021092A4
:10267000D302109250030E94B71A60938C03709398
:102680008D0380938E0390938F032196E2E00C9448
:1026900016208091F4038B7F8093F40335CF82FD65
:1026A00037CF64EF71E080E090E00E94080E88234D
:1026B00009F42ECF0E94310266E172E080E194E0DD
:1026C0000E94791C0E94F00C5D9A22CFCF93DF9379
:1026D00080E194E00E94451D892BE9F0C091D3026E
:1026E000D0E0CE0101968F7199272091D40230E07D
:1026F0008217930781F080E194E00E94721DCB5213
:10270000DD4F88838091D30290E001968F719927E5
:102710008093D302DDCFDF91CF910895A0E0B0E0A8
:10272000E4E9F3E10C94F41FD82FC62F0E94B71AE6
:102730000091A9031091AA032091AB033091AC033F
:102740006B017C01C01AD10AE20AF30A97018601E3
:1027500041E1C41647E2D406E104F10408F4D1C112
:102760006093A9037093AA038093AB039093AC0387
:1027700080910B0190910C01880F991F8093910318
:10278000892F877020919203287F282B2093920312
:1027900080910D0190910E01880F991F382F330FF2
:1027A000330F330F2770232B20939203282F22956A
:1027B0002695277080919303807C9770990F990FCD
:1027C000990F822B892B8093930320910F013091D5
:1027D0001001220F331F922F9295990F990F907C21
:1027E0008F73892B80939303932F9295990F990F51
:1027F000907C822F86958695892B8093940332FB5B
:10280000882780F9209195032E7F282B209395030C
:102810008091110190911201880F991F382F330F69
:102820002170232B20939503382F331F3327331F19
:1028300020919603207F892F8770880F232B282BC8
:10284000209396038091130190911401880F991F92
:10285000382F3295307F2F70232B20939603382FFB
:1028600032953F70209197032078892F8770829549
:10287000807F232B282B2093970380911501909123
:102880001601880F991F2F7720939703292F2795DB
:10289000222727958695822B80939803892F8695EA
:1028A0008370209199032C7F282B2093990380918A
:1028B000170190911801880F991F382F330F330F8C
:1028C0002370232B20939903382F32953695369514
:1028D000337020919A03207E892F8770880F880F8C
:1028E000232B282B20939A038091190190911A0190
:1028F000880F991F382F3295330F307E2F71232B7D
:1029000020939A039295990F907E86958695869549
:10291000892B80939B0380911B0190911C01880F50
:10292000991F80939C03892F877020919D03287F96
:10293000282B20939D0380911D0190911E01880FEB
:10294000991F382F330F330F330F2770232B20930A
:102950009D03282F22952695277080919E03807CC9
:102960009770990F990F990F822B892B80939E0353
:1029700020911F0130912001220F331F922F929539
:10298000990F990F907C8F73892B80939E03932FBF
:102990009295990F990F907C822F86958695892B19
:1029A00080939F0332FB882780F92091A0032E7F1C
:1029B000282B2093A0038091210190912201880F60
:1029C000991F382F330F2170232B2093A003382F0A
:1029D000331F3327331F2091A103207F892F877056
:1029E000880F232B282B2093A10380912301909102
:1029F0002401880F991F382F3295307F2F70232B99
:102A00002093A103382F32953F702091A2032078A4
:102A1000892F87708295807F232B282B2093A203F8
:102A20008091250190912601880F991F2F7720937F
:102A3000A203292F2795222727958695822B8093FD
:102A4000A303969593708091A4038C7F892B809328
:102A5000A4032091270130912801220F331F922FC8
:102A6000990F990F8370892B8093A4032295269543
:102A7000269523708091A503807E932F9770990FE0
:102A8000990F822B892B8093A503209129013091E6
:102A90002A01220F331F922F9295990F907E8F71EA
:102AA000892B8093A503832F8295880F807E26959E
:102AB00026952695282B2093A603DD2311F088E088
:102AC00001C080E0CC2311F094E001C090E0892B9C
:102AD0008093A7036FE070E080E194E00E94020120
:102AE000C1E9D3E0699180E194E00E949F1D83E0F9
:102AF000C83AD807B9F760E070E080E194E00E943E
:102B00000201CDB7DEB7E8E00C941020CF93C82FB8
:102B1000682F80E194E00E949F1D8C2F0E944D0140
:102B2000CF910895A0E0B0E0E8E9F5E10C94F41F3E
:102B3000C82F0E94B71A0091A9031091AA032091EF
:102B4000AB033091AC036B017C01C01AD10AE20ADD
:102B5000F30A9701860141E1C41647E2D406E10475
:102B6000F10408F445C06093A9037093AA0380930D
:102B7000AB039093AC031092BC031092BB0388EAA2
:102B80000E948615CC2311F081E801C081E00E94EB
:102B9000861580E10E94861500E010E0F801EE0F36
:102BA000FF1FE55FFE4F808191810E94F703EC01DA
:102BB000B3E0CC0FDD1FBA95E1F78D2F0E9486158B
:102BC0008C2F0E9486150F5F1F4F0031110531F7C2
:102BD0006091BC0370E080E194E00E94FA00609193
:102BE000BB037091BC03772780E194E00E94FA0058
:102BF000CDB7DEB7E8E00C941020AAE1B0E0E3E046
:102C0000F6E10C94EC1F0E949B008CE00E9487046C
:102C100081110BC06AE872E080E194E00E94791CA7
:102C200080E00E947E050E947C060E9466130E943E
:102C3000B71A0E94121091E0853009F090E01FEF62
:102C400080910204843009F494C1911192C16EC044
:102C50000E94BA0490937903809378035D9AC0929E
:102C60008C03D0928D03E0928E03F0928F0310922A
:102C70004F038091760390917703880F991F8160AD
:102C800090937703809376035E9880E00E94EF0D27
:102C90008091FE02982F9E7309F0C2C1F894809132
:102CA000E5034FEF52E06BE071E087700E9446034E
:102CB0000E94150C78949091FE028091480390FF39
:102CC000A9C1811116C0A1E5B3E080E090E0FC014C
:102CD000EE0FFF1FE55FFE4F208131812D933D9365
:102CE00001968031910599F70E94610281E08093FD
:102CF000480380915003811103C081E08093500309
:102D00001092710310927303109272038091E50385
:102D1000887109F0ADC10E94890C83E080930204A0
:102D20000E94590681E0809349035D980E94B71A7A
:102D30004B015C010E94AB1A6B017C0180914F0337
:102D4000823008F063C040908C0350908D036090F7
:102D50008E0370908F038091880390918903A091D6
:102D60008A03B0918B0384159505A605B70509F470
:102D70004DC08DEB93E00E94D4026C5D75408109DB
:102D8000910995018401041915092609370960176D
:102D9000710782079307D0F5409288035092890308
:102DA00060928A0370928B030E94B604282F80934E
:102DB0007C0380917D0390917E03820F911D9093FF
:102DC0007E0380937D0360917F036F5F60937F0339
:102DD0006930E0F070E00E94951F70937E0360936D
:102DE0007D0380917B03B3E08B9F600D711D1124E7
:102DF000769567957695679560937B030E944E0C58
:102E000010927E0310927D0310927F0380915003F5
:102E10000091D202882351F110914F03101708F04E
:102E2000A0C140908C0350908D0360908E037090F1
:102E30008F03A501940124193509460957092F8BE1
:102E4000388F498F5A8F8DEB93E00E94D4026851DE
:102E50007C4F8F4F9F4F2F89388D498D5A8D621728
:102E600073078407950708F442C27BC180918C03E5
:102E700090918D03A0918E03B0918F037501640131
:102E8000C81AD90AEA0AFB0A8DEB93E00E94D40221
:102E90009B01AC01A02FB0E00E94661F6C157D0560
:102EA0008E059F0558F480928C0390928D03A0921A
:102EB0008E03B0928F0381E0809349038091720367
:102EC000811116C08091EE03883219F40E94AD0A78
:102ED0000FC0893239F460914F03809171030E94D1
:102EE0008E1306C08A3221F4809171030E949215DC
:102EF000809149038823B9F0E0919003EF5FE0935C
:102F00009003E83131F0F0E0E354FC4F8785811104
:102F100002C010929003809190030E94A0040E942E
:102F2000E90F1092490380914E038F3F09F04BC285
:102F30000E94AB1A00914A0310914B0320914C035D
:102F400030914D03601B710B820B930B693E7340F4
:102F50008105910508F437C20E94AB1A60934A03B9
:102F600070934B0380934C0390934D030E94AC0FDE
:102F70002AC20E94B71A6B017C018091020484303E
:102F8000D1F48FE70E9465040EEF12E0E091E503B3
:102F9000E770F0E0E856FD4F808190E098012E5FE9
:102FA0003240281739070CF053CE0E947804D8011C
:102FB0008D938D01EBCFE091E503E770F0E0E856EB
:102FC000FD4F40814F5F21E0BE016F5F7F4F80E288
:102FD0000E94560A882371F010934E030E94AB1A88
:102FE00060934A0370934B0380934C0390934D037B
:102FF00090E026CEE091E503E770F0E0E856FD4F63
:10300000408150E0BE016E5F7F4F8EEF92E00E94E4
:10301000272025CE882309F46CCE1092480369CE70
:10302000982F9873983309F064CE9091F502892710
:1030300087FF5FCE90589093F5028091EE03853222
:1030400009F057CE10E0212F30E08091FE0287700A
:1030500090E0821793070CF44CCE1F5FE12FF0E055
:10306000E250FD4F608180E194E00E949F1DEBCF14
:103070008091F5029091FE02982796FD66C0807CB3
:1030800090E489278093F5028091D4023091D30295
:103090008317D1F0E6EFF2E020E02F5F90E0DC0153
:1030A000AB52BD4F4C91419301968F7199272830B7
:1030B00011F08313F2CF8093D402295C8091F50242
:1030C000282B2093F50241C080917C038093F60267
:1030D0008091E803863211F482E105C08091EB0310
:1030E000863251F48EE00E94041C95958795959543
:1030F00087958093F70202C01092F7028091EA034D
:10310000863211F483E105C08091EC03863251F4DC
:103110008FE00E94041C95958795959587958093DF
:10312000F80202C01092F80280917803909179031E
:103130009093F9028093FA0280917603909177033D
:103140009F770E9418048093FB0269E085EF92E06C
:103150000E9494060E9403078111DDCD0E94661330
:10316000F9CF10131EC080918C0390918D03A09114
:103170008E03B0918F0324013501481A590A6A0A57
:103180007B0A8DEB93E00E94D4029B01AC01A12F3E
:10319000B0E00E94661F641575058605970508F462
:1031A000DFC080914F03882309F488CE8091FE030D
:1031B0008823D9F090917103911117C04091840335
:1031C00050918503609186037091870346015701F2
:1031D000841A950AA60AB70A90E00E94360268157A
:1031E00079058A059B0508F4CFC0809100048823E7
:1031F000D9F090917303911117C0409184035091BD
:103200008503609186037091870346015701841AF4
:10321000950AA60AB70A90E00E9436026815790559
:103220008A059B0508F4C7C08091FF038823D9F065
:1032300090917203911117C04091840350918503BE
:10324000609186037091870346015701841A950A9D
:10325000A60AB70A90E00E943602681579058A0529
:103260009B0508F4ACC08091F6039091F703A09100
:10327000F803B091F903892B8A2B8B2B09F41ECE0E
:103280008091800390918103A0918203B091830388
:103290000097A105B10509F411CEC81AD90AEA0AA6
:1032A000FB0AF7FC0BCE2091FB0330E0A8EEB3E065
:1032B0000E94571F6C157D058E059F0508F0FECDF9
:1032C0008091F403829581700E946C0780E00E94D7
:1032D0007E050E9459060E94AB1A616060938003CC
:1032E000709381038093820390938303E7CD809151
:1032F000760390917703880F991F909377038093BB
:10330000760381E080934903111110C0C0928403B9
:10331000D0928503E0928603F09287031092800397
:103320001092810310928203109283031F5F109307
:103330004F038DEB93E00E94D402640D751D861D32
:10334000971D60938C0370938D0380938E039093ED
:103350008F035E9A81E00E94EF0D0E944E0C21CFF8
:10336000109277031092760381E0809349031092C4
:103370007B030E944E0C80928C0390928D03A0924E
:103380008E03B0928F030DCF81E0809371030E9472
:10339000C30C8091FA030E945B026C0D7D1D8E1D93
:1033A0009F1D61606093800370938103809382030B
:1033B000909383031ACF81E08093730335CF81E02C
:1033C0008093720350CF6A96E0E10C94082082301B
:1033D000E8F4E82FF0E0EE0FFF1FED5FFB4F718385
:1033E0006083813041F0809169008C7F842B8093D1
:1033F0006900E89A089580916900440F551F440FB1
:10340000551F837F842B80936900E99A08951F924A
:103410000F920FB60F9211242F933F934F935F9308
:103420006F937F938F939F93AF93BF93EF93FF938C
:103430008091030490910404892B29F0E091030406
:10344000F09104040995FF91EF91BF91AF919F9185
:103450008F917F916F915F914F913F912F910F903D
:103460000FBE0F901F9018951F920F920FB60F92DC
:1034700011242F933F934F935F936F937F938F9379
:103480009F93AF93BF93EF93FF9380910504909127
:103490000604892B29F0E0910504F09106040995B2
:1034A000FF91EF91BF91AF919F918F917F916F911C
:1034B0005F914F913F912F910F900FBE0F901F90F2
:1034C00018951F920F920FB60F9211242F933F93CE
:1034D0008F939F93AF93BF938091080490910904B9
:1034E000A0910A04B0910B043091070423E0230F4C
:1034F0002D3720F40196A11DB11D05C026E8230F2C
:103500000296A11DB11D2093070480930804909397
:103510000904A0930A04B0930B0480910C049091C9
:103520000D04A0910E04B0910F040196A11DB11DD0
:1035300080930C0490930D04A0930E04B0930F0499
:10354000BF91AF919F918F913F912F910F900FBE9F
:103550000F901F9018952FB7F89460910804709100
:10356000090480910A0490910B042FBF08953FB77E
:10357000F89480910C0490910D04A0910E04B091E8
:103580000F0426B5A89B05C02F3F19F00196A11D79
:10359000B11D3FBF6627782F892F9A2F620F711DAB
:1035A000811D911D42E0660F771F881F991F4A9564
:1035B000D1F70895CF92DF92EF92FF92CF93DF93EE
:1035C0006B017C010E94B71AEB01C114D104E10424
:1035D000F10479F00E94B71A6C1B7D0B683E7340B2
:1035E000A0F381E0C81AD108E108F108C851DC4F06
:1035F000ECCFDF91CF91FF90EF90DF90CF900895C7
:103600000197009739F0880F991F880F991F02972B
:103610000197F1F70895789484B5826084BD84B5EC
:10362000816084BD85B5826085BD85B5816085BDBD
:10363000EEE6F0E0808181608083E1E8F0E01082D6
:10364000808182608083808181608083E0E8F0E017
:10365000808181608083E1EBF0E080818460808301
:10366000E0EBF0E0808181608083EAE7F0E0808138
:103670008460808380818260808380818160808398
:103680008081806880831092C1000895833081F02A
:1036900028F4813099F08230A1F008958630A9F0A5
:1036A0008730B9F08430D1F4809180008F7D03C0E1
:1036B000809180008F7780938000089584B58F7704
:1036C00002C084B58F7D84BD08958091B0008F774E
:1036D00003C08091B0008F7D8093B0000895CF9398
:1036E000DF9390E0FC01E458FF4F2491FC01E05788
:1036F000FF4F8491882349F190E0880F991FFC01C6
:10370000E854FF4FA591B49182559F4FFC01C5919C
:10371000D4919FB7611108C0F8948C9120958223B1
:103720008C93888182230AC0623051F4F8948C9182
:10373000322F309583238C938881822B888304C019
:10374000F8948C91822B8C939FBFDF91CF91089539
:10375000A1E0B0E0EEEAFBE10C94F81F282F30E086
:10376000F901E859FF4F8491F901E458FF4F149192
:10377000F901E057FF4F04910023C9F0882321F09D
:1037800069830E94461B6981E02FF0E0EE0FFF1F66
:10379000E255FF4FA591B4919FB7F8948C916111B8
:1037A00003C01095812301C0812B8C939FBF21966C
:1037B000E4E00C941420CF93DF93282F30E0F9013C
:1037C000E859FF4F8491F901E458FF4FD491F90172
:1037D000E057FF4FC491CC2391F081110E94461B0A
:1037E000EC2FF0E0EE0FFF1FEC55FF4FA591B491C9
:1037F0002C912D2381E090E021F480E002C080E054
:1038000090E0DF91CF9108958E3008F08E50877050
:103810002091BB0190E4299F90011124822B809379
:103820007C0080917A00806480937A0080917A0095
:1038300086FDFCCF809178002091790090E0922B5A
:103840000895A0E0B0E0E7E2FCE10C94F41F6C0105
:103850007A01EB01E60EF71E00E010E0CE15DF0561
:1038600061F06991D601ED91FC910190F081E02D1C
:10387000C6010995080F191FF1CFC801CDB7DEB7F2
:10388000E8E00C9410206115710589F0DB010D90C2
:103890000020E9F7AD0141505109461B570BDC01EF
:1038A000ED91FC910280F381E02D0995089580E06F
:1038B00090E008950E94431C0895DC01ED91FC9175
:1038C0000190F081E02D099508950F931F93CF93F8
:1038D000DF93EC016DE00E945D1C8C016AE0CE017B
:1038E0000E945D1C800F911FDF91CF911F910F915E
:1038F00008950F931F93CF93DF93EC010E94431C15
:103900008C01CE010E94651C800F911FDF91CF9129
:103910001F910F9108950F931F93CF93DF93EC01A5
:103920000E945D1C8C01CE010E94651C800F911FBE
:10393000DF91CF911F910F910895A1E2B0E0E3EAEA
:10394000FCE10C94F01F7C01C42EE52FCB01D22E9C
:1039500019A221E02D1510F02AE0D22E8E010F5D64
:103960001F4F8D2C912CA12CB12C6C2D7E2FA501DD
:1039700094010E94A91F8C2DD29E80191124015000
:1039800011098A3010F4805D01C0895CF8018083E0
:10399000211531054105510521F0C22EE32FCA0141
:1039A000E4CFB801C7010E94431CA196ECE00C943F
:1039B0000C20A0E0B0E0EFEDFCE10C94F41FEC0172
:1039C0006A017B012115310541F4E881F9810190FB
:1039D000F081E02D642F09951DC02A303105A9F42E
:1039E00077FF12C06DE20E945D1C8C0144275527B1
:1039F000BA014C195D096E097F092AE0CE010E94C7
:103A00009D1C800F911F06C02AE0B701A601CE01C0
:103A10000E949D1CCDB7DEB7E8E00C9410200F93F8
:103A20001F93CF93DF93EC019A01AB01662757FDFB
:103A30006095762F0E94D91C8C01CE010E94651CD6
:103A4000800F911FDF91CF911F910F910895211544
:103A5000310549F4DC01ED91FC910190F081E02DFC
:103A6000642F099508950E949D1C08959A01462F80
:103A700050E060E070E00E94271D08959A01AB01BC
:103A800060E070E00E94271D0895FC0124853585C3
:103A9000F901E05CFF4F80819181F901EE5BFF4FFE
:103AA00020813181821B930B8F7399270895FC012C
:103AB00084859585FC01E05CFF4F40815181FC01CC
:103AC000EE5BFF4F208131814217530741F0019097
:103AD000F081E02DE80FF91F808190E008958FEFCD
:103AE0009FEF0895FC0184859585FC01E05CFF4F04
:103AF00040815181FC01EE5BFF4F208131814217F3
:103B0000530779F0A081B181A80FB91F8C91208152
:103B100031812F5F3F4F2F7333273183208390E014
:103B200008958FEF9FEF0895FC0181A1882329F06C
:103B3000A489B5898C9186FFFBCF11A20895CF93FC
:103B4000DF93FC0126853785D901A05CBF4F8D919D
:103B50009C91119701968F739927E901CE5BDF4FF6
:103B60004881598184179507D9F30D90BC91A02DF8
:103B7000A20FB31F6C93A685B785A05CBF4F1196AB
:103B80009C938E93A689B7892C9181E090E0078C55
:103B900002C0880F991F0A94E2F7282B2C9381E02A
:103BA00081A30488F589E02D80818064808381E091
:103BB00090E0DF91CF91089508951F920F920FB674
:103BC0000F9211242F933F934F938F939F93EF93D3
:103BD000FF938091C00082FD1CC04091C60080917F
:103BE000B6049091B70401968F7399272091B80479
:103BF0003091B9048217930771F0E091B604F09107
:103C0000B704EA58FB4F40839093B7048093B604FF
:103C100002C08091C600FF91EF919F918F914F91CB
:103C20003F912F910F900FBE0F901F90189580E13C
:103C300094E00E94451D892B11F00E94DC1D08951F
:103C40001F920F920FB60F9211242F933F938F93D1
:103C50009F93EF93FF9320917204309173048091AE
:103C60007404909175042817390731F48091C100CC
:103C70008F7D8093C10014C0E0917404F0917504AD
:103C8000EE5CFB4F20818091740490917504019645
:103C90008F73992790937504809374042093C600C2
:103CA000FF91EF919F918F913F912F910F900FBEB8
:103CB0000F901F901895A0E0B0E0E1E6FEE10C94B3
:103CC000F01FFC011382128288EE93E0A0E0B0E0C6
:103CD00084839583A683B78384EC92E09183808369
:103CE0007587648757874687318B208B138B028BB0
:103CF000F58AE48AD78AC68AB18EA08E938E828E88
:103D00008F85848F8889858F8989868F8A89878F17
:103D10008B8980A3ECE00C940C20CF92DF92EF9281
:103D2000FF92CF93DF93EC016A017B01411581EE95
:103D3000580761057105F9F0EC89FD8981E090E093
:103D400008A002C0880F991F0A94E2F7808360E000
:103D500079E08DE390E0A70196010E94A91F215010
:103D600031094109510956954795379527952115F0
:103D700080E1380798F0EC89FD89108260E874E8EA
:103D80008EE190E0A70196010E94A91F2150310900
:103D9000410951095695479537952795E889F9893D
:103DA0003083EA89FB89208319A2EE89FF8940814B
:103DB00081E090E09C010C8C02C0220F331F0A941A
:103DC000E2F7422B4083EE89FF8940819C010D8CF4
:103DD00002C0220F331F0A94E2F7422B4083EE8980
:103DE000FF8940819C010E8C02C0220F331F0A9470
:103DF000E2F7422B4083EE89FF8920810F8C02C0BD
:103E0000880F991F0A94E2F7809582238083DF91BF
:103E1000CF91FF90EF90DF90CF9008958F929F9277
:103E2000AF92BF92CF92DF92EF92FF920F931F93C8
:103E300081E08F9385E08F9387E08F9383E08F936A
:103E400084E08F93E6EC8E2E912CF2ECAF2EB12C09
:103E5000A1ECCA2ED12CB0ECEB2EF12C04EC10E02E
:103E600025EC30E042E354E066E774E080E194E062
:103E70000E945B1E0F900F900F900F900F901F915C
:103E80000F91FF90EF90DF90CF90BF90AF909F90F9
:103E90008F9008950E940B1B0E940712C7E1DEE17C
:103EA0000E94FD152097E1F30E94171EF9CFA29FF3
:103EB000B001B39FC001A39F700D811D1124911DFE
:103EC000B29F700D811D1124911D08950E94571FEE
:103ED000A59F900DB49F900DA49F800D911D11245E
:103EE0000895B7FF0C94661F0E94661F821B930BF8
:103EF0000895DB018F939F930E94661FBF91AF913E
:103F0000A29F800D911DA39F900DB29F900D112433
:103F10000895991B79E004C0991F961708F0961B25
:103F2000881F7A95C9F780950895AA1BBB1B51E19C
:103F300007C0AA1FBB1FA617B70710F0A61BB70B19
:103F4000881F991F5A95A9F780959095BC01CD01BE
:103F50000895A1E21A2EAA1BBB1BFD010DC0AA1FCA
:103F6000BB1FEE1FFF1FA217B307E407F50720F0E2
:103F7000A21BB30BE40BF50B661F771F881F991F5D
:103F80001A9469F760957095809590959B01AC01A6
:103F9000BD01CF010895052E97FB1EF400940E94E9
:103FA000E21F57FD07D00E94A91F07FC03D04EF463
:103FB0000C94E21F50954095309521953F4F4F4FFF
:103FC0005F4F089590958095709561957F4F8F4FC5
:103FD0009F4F08952F923F924F925F926F927F92E0
:103FE0008F929F92AF92BF92CF92DF92EF92FF9209
:103FF0000F931F93CF93DF93CDB7DEB7CA1BDB0BB5
:104000000FB6F894DEBF0FBECDBF09942A88398859
:1040100048885F846E847D848C849B84AA84B98460
:10402000C884DF80EE80FD800C811B81AA81B9816C
:10403000CE0FD11D0FB6F894DEBF0FBECDBFED0180
:104040000895EE0FFF1F0590F491E02D0994FB01F8
:10405000DC0102C001900D9241505040D8F7089504
:10406000F999FECF92BD81BDF89A992780B5089540
:10407000262FF999FECF1FBA92BD81BD20BD0FB684
:10408000F894FA9AF99A0FBE01960895F894FFCF22
:104090000000BA04200008409C88130002000200BF
:1040A0000200020002000200020002000200020000
:1040B000020002000200020002000280250000054A
:1040C000400AA1204EA50020244EA52C2330C0126A
:1040D00000001A400AA1204EA5001B1E27522C23C7
:1040E000308025000005400AA1204EA50020244E66
:1040F000A52C2330004B000006400AD0009D49004B
:104100007B289D492C233000E1000005400A450131
:10411000D7DC03B81E0EBF00232E48E801008A40FA
:104120000A6001555502AD1E20000023C800200181
:104130002201260221022703230326042605260541
:104140002B0624072507280729072A01545820741D
:10415000696D656F7574210057616974696E6720B8
:1041600062696E640A00476F7420706B740A0064A1
:1041700061746120676F6F640A007363616E6E65BE
:1041800072206D6F6465004F70656E4C52536E67A0
:10419000205258207374617274696E672000206F1A
:1041A0006E204857200053617665642062696E6412
:1041B000206461746120746F20454550524F4D0A50
:1041C000004920616D20736C61766500456E7465F1
:1041D00072696E67206E6F726D616C206D6F6465C1
:1041E00000454550524F4D2064617461206E6F74DC
:1041F0002076616C6964206F722062696E64206A47
:10420000756D70706572207365742C20666F7263B3
:10421000696E672062696E640A0052582068616E98
:104220006700B200F4014C0300070B0C10111500DD
:10423000091203130E0F000102000000100000001D
:104240000800200000010000020000000100000240
:10425000000000009F1D211C451D721D571D941D4F
:107E00000F92CDB7DEB7112484B714BE81FFF1D035
:107E100082E08093C00088E18093C10086E0809377
:107E2000C20080E18093C4008EE0CDD088249924E4
:107E3000CC24C394F5E0DF2EE1E1EE2E73E0F72EC3
:107E4000B6D0082F813479F4B2D08983C2D0898129
:107E5000823811F481E005C0813811F485E001C059
:107E600083E09ED09AC0823411F484E103C085344B
:107E700019F485E0B6D091C0853561F498D0082F0B
:107E800010E095D090E0982E8824802A912A880CC2
:107E9000991C82C0863521F484E0A3D080E0E1CF34
:107EA000843609F04CC083D082D0A82E80D0B82E62
:107EB00000E011E07CD0F80181938F01AE16D1F77C
:107EC00088D0FB2DF53489F4E0E0F1E00BC0F9999E
:107ED000FECF92BC81BC0894811C911C819180BD15
:107EE000FA9AF99AEA1598F358C08B2D863409F05E
:107EF00054C0F401F7BEE89507B600FCFDCFF401CD
:107F0000A0E0B1E02C9130E011968C91119790E0B7
:107F1000982F8827822B932B12960C01C7BEE895C9
:107F20001124329681E0A038B80761F7F401D7BE7A
:107F3000E89507B600FCFDCFE7BEE8952EC0843774
:107F4000F1F435D034D0182F32D0B82E42D0FB2DDA
:107F5000F63421F4F40105914F010CC0FB2DF534EA
:107F600049F4F999FECF92BC81BC0894811C911C04
:107F7000F89A00B5802F14D0115049F70EC08537FC
:107F800039F427D08EE10CD085E90AD08FE069CF93
:107F9000813511F488E017D01CD080E101D050CF9A
:107FA0009091C00095FFFCCF8093C600089580910A
:107FB000C00087FFFCCF8091C00084FD01C0A89560
:107FC0008091C6000895E0E6F0E098E19083808318
:107FD0000895EDDF803219F088E0F5DFFFCF84E10E
:107FE000DFCF1F93182FE3DF1150E9F7F2DF1F9166
:0E7FF0000895282E80E0E7DFEE27FF27099492
:027FFE0001057B
:0400000300007E007B
:00000001FF
